:020000040000FA
:10000000590A490852084308760831082E08310871
:100010005008200862087908200841086C08650823
:10002000780841084C084208200861086C086208FA
:100030004008630872086F08770864082E08720881
:1000400075082008280843082908430852084F0863
:10005000570844082008520875087308730869088F
:1000600061082C082008500865086E087A086108A5
:0A007000200832083008300832087A
:04007A000008000872
:02007E00270059
:100080000400080C2800E802430A0400E702410AC1
:100090000008270004008605040C2800E8024E0A28
:1000A0008604030C2800E802530A0400E7024B0A06
:1000B000000825000F0C02002F0C06008604E30741
:1000C0006B0A6F0004000607710A26077A0A6607A2
:1000D000830AEF02620A06020B0E0B0F4307610A46
:1000E00003007B0C2B00D50C2C000B0C2D00160CE8
:1000F0002E008C0A7B0C2B00D50C2C00210C2D0023
:100100002C0C2E008C0A7B0C2B00D50C2C00370CF1
:100110002D00420C2E008C0AFA0C4909410C4909A9
:10012000A50C3F09040C29000B0C2400080C2A0024
:10013000220C4909220C3F09220C200303063F0927
:10014000EA02980AA402E902960A220C49090D0C57
:0C0150002900FF0C3F09E902A90A610A1E
:0203FE00700C81
:021FFE00EE0FE4
:00000001FF
